:1000000044C053C052C051C050C04FC041C14DC088
:100010004CC04BC04AC03BC266C247C046C045C088
:1000200044C043C042C04261747465727920566F07
:100030006C746167653A202020006D560D0A0047F8
:10004000656E657261746F7220566F6C746167655E
:100050003A202020006D560D0A0047656E657261DA
:10006000746F723A20006D41202000570D0A007312
:100070007769746368657320286C6F61642C2067EE
:10008000656E293A20000D0A000011241FBECFE53D
:10009000D4E0DEBFCDBF10E0A0E6B0E001C01D920D
:1000A000A53BB107E1F79BD246C3AACFCF9364E04B
:1000B00082E044D1CFE09C01C29FC001C39F900D5C
:1000C00011248A5E9C4F90936B0080936A0064E0D9
:1000D00080E034D19C01C29FC001C39F900D1124C8
:1000E000909369008093680064E081E027D18F5F7E
:1000F000914097FD05C090936F0080936E0004C0FF
:1001000010926F0010926E0020916E0030916F007F
:1001100048E4429FC001439F900D112490936700D3
:1001200080936600CF910895CF93DF93EC01CB01CC
:1001300024E630E0B901ECD2FB01CE01B901D4D202
:10014000E69FC001E79F900DF69F900D1124B90125
:10015000CBD2CB01DF91CF91089586E290E032D2ED
:1001600080916A0090916B005DD18AE390E02AD281
:100170008FE390E027D2809168009091690052D17E
:1001800085E590E01FD28AE590E01CD28091660060
:100190009091670047D186E690E014D28091660086
:1001A0009091670024E630E0B901B2D2FB01809162
:1001B0006A0090916B00B90197D2E69FC001E79F5A
:1001C000900DF69F900D1124B9018ED2CB012AD14A
:1001D0008BE690E0F7D18FE690E0F4D186B38170A2
:1001E000805DD4D18CE2D2D186B386958170805D5A
:1001F000CDD186E890E0E6C180916A0090916B00D5
:10020000803C9B4250F410926200809163008530E4
:1002100068F48F5F8093630009C01092630080913F
:100220006200833018F48F5F8093620080916800D1
:1002300090916900893C924350F010926000809147
:100240006100833068F48F5F8093610009C0109271
:10025000610080916000811103C081E080936000A3
:1002600080916300853018F0109262000FC0809179
:100270006200833060F010926300809161008330EF
:1002800010F0C09A0895809160008111C09808957F
:100290001F920F920FB60F9211242F933F934F93FB
:1002A0005F936F937F938F939F9380916C00909156
:1002B0006D00019690936D0080936C0020916C000E
:1002C00030916D0081E090E020364AEE340710F462
:1002D00080E090E060E67AEE869FA001879F500D57
:1002E000969F500D1124C901841B950B90936D00AE
:1002F00080936C009F918F917F916F915F914F914F
:100300003F912F910F900FBE0F901F90189580E492
:1003100087B983E086B9379A369A3699FECF84B189
:1003200095B1089597B18F71907E892B87B9369AD0
:100330003699FECF24B135B1C9010895FF920F93CC
:100340001F93CF93DF93082F862F6CE3C1D1F92E33
:1003500010E0C0E0D0E005C0802FE4DFC80FD91F57
:100360001F5F1F11F9CF612FCE0170E0BDD1CB010E
:10037000DF91CF911F910F91FF900895811101C0DE
:1003800084E690E0EFE1FEE43197F1F700C0000071
:100390009F5F9813F7CF0895EF92FF920F931F93EB
:1003A000CF93DF938C0160E177E29ED17C01862FB1
:1003B000805DECD0C8EED3E0C701BE0195D1862F99
:1003C000805DE4D08EE2E2D0C801BE018DD164E64A
:1003D00070E08AD1862F805DDF91CF911F910F91C0
:1003E000FF90EF90D3C00F931F93CF93DF931F9293
:1003F000CDB7DEB7082F64E66BD1805D9983C6D098
:100400001AE09981892F612F63D1805DBFD0802F41
:10041000612F5ED1892F805D0F90DF91CF911F9169
:100420000F91B4C0EF92FF920F931F93CF93DF937E
:10043000EC0160E177E258D17C01862F805DA6D087
:1004400008EE13E0C701B8014FD1862F805D9ED022
:10045000CE01B80149D104E610E0B80145D1862F9C
:10046000805D94D0CE01B8013FD10AE010E0B80120
:100470003BD1862F805D8AD0CE01B80135D1805D19
:10048000DF91CF911F910F91FF90EF907FC01F924E
:100490000F920FB60F9211242F938F939F93EF9388
:1004A000FF938BB19CB18871E0917200EF5FEF71A7
:1004B00020917100E21739F0E0937200F0E0EB5800
:1004C000FF4F908301C082E090917000982B909331
:1004D0007000FF91EF919F918F912F910F900FBE20
:1004E0000F901F9018951F920F920FB60F92112424
:1004F0008F939F93EF93FF9390917400809173007B
:10050000981761F0E0917300EF5FEF71E093730073
:10051000F0E0EB56FF4F80818CB901C05598FF91F8
:10052000EF919F918F910F900FBE0F901F90189594
:100530001092740010927300109272001092710069
:1005400097FF03C022E02BB99F7790BD89B988E956
:100550008AB986E880BD08959091720080917100FB
:10056000981781F0E0917100EF5FEF71E0937100F7
:10057000F0E0EB58FF4F20818091700010927000E6
:1005800030E002C020E031E0C9010895909174008C
:100590009F5F9F71209173009217E1F3E92FF0E0C4
:1005A000EB56FF4F808390937400559A0895CF9334
:1005B000DF93EC0101C0EADF89918111FCCFDF916B
:1005C000CF910895CF93DF93EC0101C0DFDFFE01EF
:1005D000219684918111FACFDF91CF91089587B34D
:1005E000836087BB88B38C7F88BB91DE8EB58B60C0
:1005F0008EBD82EE94E09BBD8ABD80E189BF789478
:1006000089E190E095DFC098C19AC4E6D0E080917E
:100610006C0090916D008436910530F010926D0061
:1006200010926C0043DDE8DD97DF811521E0920731
:1006300071F399278136910529F08037910539F7B3
:100640008CDDE5CF81E4A2DF80916A0090916B00A0
:10065000E9DE8CE29BDF8091660090916700E2DE2C
:100660008CE294DF80E090E0DDDE8CE28FDF809131
:10067000660090916700BE014BD09B0180916A009B
:1006800090916B00BE0130D0269FC001279F900D36
:10069000369F900D1124BE0127D0CB01C3DE8CE222
:1006A00075DF80E090E0BEDE8CE270DF86B38170A3
:1006B000805D6CDF8CE26ADF80E368DF8CE266DFFE
:1006C00086B386958170805D61DF82E45FDF9FCFB6
:1006D000991B79E004C0991F961708F0961B881F94
:1006E0007A95C9F780950895AA1BBB1B51E107C0F5
:1006F000AA1FBB1FA617B70710F0A61BB70B881FB2
:10070000991F5A95A9F780959095BC01CD01089540
:1007100097FB072E16F4009406D077FD08D0E4DF8F
:1007200007FC05D03EF4909581959F4F08957095F4
:0A07300061957F4F0895F894FFCF04
:00000001FF
